:020000040000FA
:020000000828CE
:020008000900ED
:10001000203084008001840A60300402031C0A2816
:100020002A16FF30C200831685018515831207301A
:100030009900C030831681008312313090008E0108
:100040008F0100308B00003083168C0083128316E2
:1000500031309B001C141A088312C500163045026B
:10006000031C3328C501640085193B280A30C207E8
:10007000031842284A2841184A280A30C202031CA1
:1000800046284A284110FF30C2004A284114C201C4
:100090003B214A288F08031933288F01003045027D
:1000A000031D5A283F10BF103F135321AF21C22117
:1000B000DD21F02101304502031D66283F10BF10ED
:1000C0003F135321AF21C2211822F02102304502F3
:1000D000031D72283F10BF103F135321AF21C221CF
:1000E000DD21632203304502031D7E283F10BF102F
:1000F0003F135321AF21C22118226322043045024D
:10010000031D8A283F10BF103F175321AF21C22182
:10011000DD21F02105304502031D96283F10BF1058
:100120003F175321AF21C2211822F021063045028A
:10013000031DA2283F10BF103F175321AF21C2213A
:10014000DD21632207304502031DAE283F10BF109A
:100150003F175321AF21C2211822632208304502E4
:10016000031DB9283F10BF103F175321AF21302284
:10017000F02109304502031DC4283F10BF103F176E
:100180005321AF21302203220A304502031DCE281D
:100190003F14BF103F1753213022F0210B3045028E
:1001A000031DD8283F14BF103F17532130220322CC
:1001B0000C304502031DE3283F14BF103F175321A5
:1001C000C221DD21F0210D304502031DEE283F1430
:1001D000BF103F175321C2211822F0210E304502D3
:1001E000031DF9283F14BF103F175321C221DD2101
:1001F00063220F304502031D04293F14BF103F172F
:100200005321C2211822632210304502031D0E29FA
:100210003F14BF143F175321C221F0211130450272
:10022000031D18293F14BF143F175321C221032275
:1002300012304502031D22293F14BF143F175321DA
:10024000C221632213304502031D27298D2114305A
:100250004502031D31293F14BF143F176E21DD21D4
:10026000F02115304502031D3A293F14BF143F17F2
:100270006E2121223328C50A16304502031C33287B
:10028000C5018B13450883161C159A0031309B005D
:1002900055309D00AA309D009C149C184D291C11BE
:1002A00083128B170800B00A0A303002031C0800C2
:1002B000B11C8512B1180512F530311C2D303002F9
:1002C000031C0800B10A3F1CB11001303F1FB100F0
:1002D000B11C8516B1180516B0010800B00A0A3025
:1002E0003002031C08008512051205111E30B118DA
:1002F0005030311958303002031C08000310B10D82
:10030000B1193114B1080319311431188516B11817
:10031000051631190515B0010800B00A0A3030027F
:10032000031C0800851205120511851005107D308B
:10033000311C53303002031C0800B10A0330B105F0
:10034000B1080319851603190516B1180515B1185A
:1003500085143118AD29B1180514B0010800B20A8E
:100360000A303202031C08000512FF30331C3730FC
:100370003202031C0800B30A01303F1FB300051608
:10038000B2010800B40A0A303402031C0800B51C8C
:100390000511B51885107830351C32303402031C35
:1003A0000800B50ABF1CB51001303F1FB500B51CD1
:1003B0000515B5188514B4010800B60A0A303602CE
:1003C000031C08008510C830381C1E303602031C80
:1003D0000800B80A01303F1FB8008514B6010800B4
:1003E000B90A0A303902031C08000510F0303A1C23
:1003F00028303902031C0800BA0A01303F1FBA0036
:100400000514B9010800B90A14303A1C4630390203
:10041000031C0800051064303A1C6E303902031CBE
:100420000800BA0A01303F1FBA000514B9010800DC
:100430003608B60B08000508023A8500C830B60039
:1004400008003608B60B0800B70A371C0800050874
:10045000023A85000510851C0514A030B60008007E
:10046000A80F382AA80A0310AA0DAA1AAA15AA12B8
:10047000FC22AB001330AA19AB0268302A0503191D
:10048000432A851005152A132B080E0203184E2A3D
:1004900014302A0503194E2A851405118F08031DEF
:1004A000080064002B080E02031C4E2A14302A0593
:1004B00003195C2A8510051528302A050319622ABC
:1004C000851405110800A80F6B2AA80A0310AA0DAD
:1004D000AA1AAA15AA12FC22AB001330AA19AB0261
:1004E00068302A05031D05102A132B080E02031875
:1004F0007D2A14302A05031D05148F08031D0800EA
:1005000064002B080E02031C7D2A14302A05031DEB
:0C051000051028302A05031D0514080002
:0805F80003308A00280382078A
:10060000143417341B341E342134253428342B344D
:100610002E343134343437343A343D344034423477
:10062000453448344B344D345034523455345734B7
:100630005A345C345F3461346334663468346A3409
:100640006C346F34713473347534773479347B346B
:100650007D347F34813483348434863488348A34DE
:100660008C348D348F34913492349434963497345E
:1006700099349A349C349D349F34A034A234A334EA
:10068000A434A634A734A834AA34AB34AC34AE3482
:10069000AF34B034B134B234B434B534B634B73422
:1006A000B834B934BA34BB34BC34BD34BE34BF34CE
:1006B000C034C134C234C334C434C534C634C7347E
:1006C000C834C934CA34CA34CB34CC34CD34CE3433
:1006D000CE34CF34D034D134D134D234D334D434F2
:1006E000D434D534D634D634D734D834D834D934B5
:1006F000DA34DA34DB34DB34DC34DD34DD34DE347C
:10070000DE34DF34DF34E034E034E134E134E23449
:10071000E234E334E334E434E434E534E534E63419
:10072000E634E734E734E734E834E834E934E934EC
:10073000EA34EA34EA34EB34EB34EB34EC34EC34C2
:10074000EC34ED34ED34EE34EE34EE34EF34EF349B
:10075000EF34EF34F034F034F034F134F134F13478
:10076000F134F234F234F234F334F334F334F33456
:10077000F434F434F434F434F534F534F534F53435
:10078000F534F634F634F634F634F734F734F73417
:10079000F734F734F834F834F834F834F834F834FB
:1007A000F934F934F934F934F934FA34FA34FA34DE
:1007B000FA34FA34FA34FA34FB34FB34FB34FB34C5
:1007C000FB34FB34FB34FC34FC34FC34FC34FC34AC
:1007D000FC34FC34FC34FD34FD34FD34FD34FD3494
:1007E000FD34FD34FD34FE34FE34FE34FE34FE347C
:0E07F000FE34FE34FE34FE34FE34FF34FF349B
:084000000000010000000900AE
:02400E00CC01E3
:00000001FF
